:10000000FB3065000030660088280E087F398207C3
:100010000034003400340034003400340034003440
:100020000034003400340034003400340034003430
:10003000713477346534723474347A347534693495
:100040006F347034FCFF2B3400340034003400343F
:100050006134733464346634673468346A346B34BE
:100060006C34F6FFE4FF0034003400340034003414
:1000700000340034003400340034003400340034E0
:1000800000340034003400340034003400340034D0
:1000900000340034003400340034003400340034C0
:1000A00000340034003400340034003400340034B0
:1000B00000340034003400340034003400340034A0
:1000C0000034003400340034003400340034003490
:1000D0000034003400340034003400340034003480
:1000E0000034003400340034003400340034003470
:1000F0000034003400340034003400340034003460
:10010000003400340034003400340034003400344F
:100110008E010B300E0203199F2892208F00D620EB
:100120008E0A89280E0882076D346134633468347E
:100130006534203452344534533445345434B22079
:1001400007308C00CD208E0D8C0BA2288E0DCD207B
:100150008E0C8E090530BA2005208F008E1FD62008
:10016000C320A028CD20FA30BA20CD200130BA20FB
:10017000C32008008C00F8308D0000008D0BBD28D6
:100180008C0BBB280800F9306500851028308C00E6
:100190008C0BC828FB30650008000518CD28851C8D
:1001A000031085180314051CD3280800E720E72056
:1001B000051508308C008F09E7208F0C031C0511F2
:1001C000031805158C0BDC28E720051108000D30FD
:1001D0008D008D0BE92800000800FF3FFF3FFF3F27
:10400000FF3FFF3FFF3FFF3FFF3FFF3FFF3FFA3FC5
:00000001FF
